:1000000000308A00AB2900000F080E3C031D0B28AE
:1000100060308D007D290F08163C031D12283130F9
:100020008D007D290F081E3C031D192832308D00DC
:100030007D290F08263C031D202833308D007D29A3
:100040000F08253C031D272834308D007D290F081B
:100050002E3C031D2E2835308D007D290F08363C9F
:10006000031D352836308D007D290F083D3C031DCA
:100070003C2837308D007D290F083E3C031D432866
:1000800038308D007D290F08463C031D4A28393041
:100090008D007D290F08453C031D512830308D000F
:1000A0007D290F084E3C031D58282D308D007D29D9
:1000B0000F08553C031D5F283D308D007D290F083A
:1000C0005D3C031D66285C308D007D290F08663C71
:1000D000031D6D2858308D007D290F080D3C031D30
:1000E000742854308D007D290F08153C031D7B2892
:1000F00071308D007D290F081D3C031D822877304B
:100100008D007D290F08243C031D892865308D0052
:100110007D290F082D3C031D902872308D007D290C
:100120000F082C3C031D972874308D007D290F0883
:10013000353C031D9E2879308D007D290F083C3CFD
:10014000031DA52875308D007D290F08433C031D34
:10015000AC2869308D007D290F08443C031DB3286D
:100160006F308D007D290F084D3C031DBA2870307B
:100170008D007D290F08543C031DC1285B308D0084
:100180007D290F085B3C031DC8285D308D007D294B
:100190000F08583C031DCF2843308D007D290F08E0
:1001A0001C3C031DD62861308D007D290F081B3CA7
:1001B000031DDD2873308D007D290F08233C031DAE
:1001C000E42864308D007D290F082B3C031DEB28AB
:1001D00066308D007D290F08343C031DF2286730FE
:1001E0008D007D290F08333C031DF92868308D00F0
:1001F0007D290F083B3C031D00296A308D007D29B5
:100200000F08423C031D07296B308D007D290F0824
:100210004B3C031D0E296C308D007D290F084C3C92
:10022000031D15293B308D007D290F08523C031D0D
:100230001C2927308D007D290F085A3C031D2329D6
:100240000A308D007D290F08123C031D2A295330E6
:100250008D007D290F081A3C031D31297A308D004D
:100260007D290F08223C031D382978308D007D2917
:100270000F08213C031D3F2963308D007D290F08A5
:100280002A3C031D462976308D007D290F08323C1B
:10029000031D4D2962308D007D290F08313C031D5F
:1002A00054296E308D007D290F083A3C031D5B29CF
:1002B0006D308D007D290F08413C031D62292C30D3
:1002C0008D007D290F08493C031D69292E308D00C2
:1002D0007D290F084A3C031D70292F308D007D2990
:1002E0000F08593C031D772953308D007D290F08D5
:1002F000293C031D7D2920308D00AD2A8316051170
:100300008312051109308D000000000000008D17D8
:100310009A298D130E0D0D0B900C03180515031C57
:1003200005110D179A290D138D0B8A290000000065
:100330000000051501308C008401840B9D298C0B75
:100340009C290D308400840BA32900008D1B892972
:100350000D1B9329BA2A84011F3083058E01831651
:1003600005118312051508308C008C1DBF2907303C
:100370008101813084000008C0390F38800064009A
:10038000813084000008C0390C0480008F0183167E
:10039000051483120518CD29C72983160514831265
:1003A000051CD329CD298316051483120518D929D4
:1003B000D329831605148312051CDF29D929831636
:1003C000851400308312851801308F0483160514BC
:1003D00083120518EC29E629831605148312051CDF
:1003E000F229EC2983168514003083128518013018
:1003F0008C0003108C0D0C088F04831605148312D7
:100400000518032AFD29831605148312051C092AE1
:10041000032A8316851400308312851801308C005E
:100420008C0D8C0DFC308C050C088F048316051484
:10043000831205181C2A162A831605148312051C1C
:10044000222A1C2A83168514003083128518013055
:100450008C008C0D8C0D8C0DF8308C050C088F04E5
:100460008316051483120518362A302A83160514BC
:100470008312051C3C2A362A831685140030831209
:10048000851801308C008C0EF0308C050C088F0420
:1004900083160514831205184E2A482A831605145C
:1004A0008312051C542A4E2A8316851400308312A9
:1004B000851801308C008C0E8C0DE0308C050C08FA
:1004C0008F048316051483120518672A612A831680
:1004D00005148312051C6D2A672A831685140030C3
:1004E0008312851801308C008C0E8C0D8C0DC03061
:1004F0008C050C088F048316051483120518812AB5
:100500007B2A831605148312051C872A812A8316E9
:10051000851400308312851801308C000C0C8C017E
:1005200003188C170C088F04831605148312051802
:100530009A2A942A831605148312051CA02A9A2A43
:100540008316051483120518A62AA02A83160514FB
:100550008312051CAC2AA62A04280D088F000F0858
:10056000F03C0319BA2A0F08733C0319BA2A0F0882
:0805700090007E29C6296300FA
:02400E00F93F78
:00000001FF
